:020000040000FA
:04000000000078285C
:08000800F100030E8301F20078
:100010000A08F3008A110A120B1D4A280B11351E1B
:100020001F280830860624308100FA0B70288611BC
:100030008316031387308100831203133512B51919
:10004000702887253F3A03193F2875087402031D5D
:100050003328F70B7028B5183128791B3128B514CF
:100060003328B5107917FB1C452835168316031362
:1000700083308100831203139630FA0045287508F7
:100080007402031970287408F6007508F4004C30E7
:10009000F70070280D1C70280D10351C70281D1CD1
:1000A00059281B08C3001C08C4009D0104309D0092
:1000B000702843089B02031C9C0311301B02031C85
:1000C0009C03C30044089C0227301C02C400871D07
:1000D000C4178030C018C4069D0105309D0035103E
:1000E000830173088A00720E8300F10E710E0900FD
:1000F000831203138B018A01850186018701C001E8
:10010000B501FC01FE240530C2001030F9003F307B
:10011000F400F6004C30F70007308A008316031312
:100120008E309F00C13085008312031381309F0001
:1001300083160313C0308600CB30870087308100E0
:1001400083120313033090009D0105309D00831638
:10015000031313309900B0309800831203139030CA
:100160009800A9258A110A16F1228A110A1283160B
:10017000031301308D0083120313E0308B004230F3
:100180001726542583120313F80A0A30780203193C
:10019000F8013F3076020319B329791FDC2879135F
:1001A000F61AD7283F30F6008A110A16A129761AC6
:1001B000DC280230FB06AE29B51C1B29B510761AC7
:1001C000E4280130FB06B329F61AE9284030B506C9
:1001D000B329F619EE282030B506B3297618FF2882
:1001E0000130FC067C1C3C29E3247B15D02594308F
:1001F00017269A301726D425AB301726B32976193F
:1002000009297D1C06297D10FD14AE297D14FD10E1
:10021000AE29F618B3292030FC06FC1E3C29E32445
:10022000D02594301726A53017264208ED25D42571
:10023000AB301726B329FC1A3029351B7D297C1CCD
:100240004029761830290430FB06D0259430172633
:100250009A307B1D9F301726D425AB301726B32943
:10026000F6183C297B14FB13C1016324F8017C18A8
:10027000FC14FC1A7C17B3297C10FC12F024B3295F
:1002800076184929C10A4108033C0319C1016324B6
:10029000AE29F6184E290430FB06AE2976195929E5
:1002A00003307D057D10FD10031DAE290830FB06CF
:1002B000AE29F619662960307B05403C031D632991
:1002C0009F30FB05AE292030FB07AE29761A722934
:1002D0007B1C6C297B10B329C20A4208083C031915
:1002E000C201B329F61AB3298030FB06FB1FB329DC
:1002F000CE30D5254830EF25B329761880294229FC
:10030000F6188D290C3079050C3C031D8A29F33031
:10031000F905B3290430F907B32976199A2903306E
:100320007905033C031D9729FC30F905B3290130F9
:10033000F907B329F619A72930307905303C031D98
:10034000A429F9127916B3291030F907B329761ABE
:10035000B3290230C00640080508B3298A110A16DD
:1003600003238A110A123F30F600FC18C4297C1BB3
:10037000C429351B8F2A7C18C129FC1AC129FB1FEF
:10038000C42966256625C928FC139C24C010400892
:1003900085000716A0305324F8210038031DC92812
:1003A0000712B4305324F8210038031DC92807224E
:1003B0000038031DC928B424C0144008850007165E
:1003C000C8305324F8210038031DC9280712DC3037
:1003D0005324F8210038031DC92807220038031DC3
:1003E000C9289C24C01040088500071631229C2A89
:1003F00044087F394E3A031D00344308213A031D57
:100400000034FC177B1C0034C01C202A2C2AA0308E
:10041000C018C83084000310780D013E84077F3077
:100420000005063C031C0034143084077F300005AF
:10043000063C031C00347B1C0034C01C2C2A202AE0
:100440000730420203190034C20ACE30D5254130AC
:10045000EF254208ED250134C20803190034C20318
:10046000252A0430CC000930F808031D7803CA009F
:100470000310CA0DA030CA07A030CB000310780DBE
:10048000CB074B0884000008A600840A0008A700D8
:100490004A0884000008AD00840A0008AE008030DD
:1004A000AE06273073222E30732288227F22FF303F
:1004B000AE00E230AD008822A71F0A2D1430CA0713
:1004C000CB07CC0B412A7D1D672AFD19080004309B
:1004D000FD077D1D0800FD1D08008A110A168321F5
:1004E0008A110A1208008400801F08008013800906
:1004F00084038009800F0800840A800A0800A71F6F
:1005000008000130A602031CA703A609A7090800DA
:100510002D08A6072E0803182E0FA7070800C124D0
:10052000F801791E962A0716A0305324F91EDE2BF7
:100530000712B4305324DE2BA030E1005130E0002C
:100540002425B430E1005530E0002425C830E10016
:100550005930E0002425DC30E1005D30E000242546
:10056000030159045D040319B32BFC1BB32B420890
:10057000CA000310CA0DCA0D8A150A1200304A07B4
:10058000BA2561300C2651301126592151300C26E4
:100590006130142655301126592155300C268A1108
:1005A0000A127C1FD62A8A110A16F22C8A110A1204
:1005B000FC1CE02A8A150A128E258A110A12222CA6
:1005C0008A150A128E258A110A128A150A125625D0
:1005D0008A150A1244268A110A12B51AB92BD02597
:1005E00060307B0503191B2B203C031D092B513068
:1005F000EF25EB258A150A125530142651301126A5
:10060000B7217F30A7058A110A123130FE005D261E
:10061000412B4430EF25EB258A150A125130142660
:1006200055301126B7217F30A7058A110A123430C0
:10063000FE005D26412B7B1D282B17308A150A12E0
:10064000262651301126B72151300C268A110A1264
:100650005230EF25A3230B308A150A12262651307B
:100660001126AE134C238A110A12013C03193B2BAD
:10067000BB301726412B3430FE0051305626013056
:10068000EF25C90E7B1D512B17308A150A1226261D
:1006900055301126B7218030A70655300C268A1117
:1006A0000A120310410DCA00CA0DCE304A078A153E
:1006B0000A1226268A110A12D425FB1D692B5830EE
:1006C000EF25A3233430FE00553056260130EF25A8
:1006D0008D2BF91F7D2B8030D4068A150A125530D8
:1006E0001126B7218A110A124330EF25A323A9232B
:1006F000DB265D264630EF258D2B8A150A125530F4
:10070000112659218A110A124C30EF25A323A9235F
:10071000E0265D264830EF258D2B8D30D52517241A
:100720007B1C962BCE30D5254130EF25CF30D525FB
:100730004208ED258A110A161A258A150A12C926B9
:100740008A110A12C22870307B1D7330EF25EB2509
:10075000080003307D05031D0800C230D525073091
:10076000EF25EB250800B51AB92BD02565301726E3
:100770008D2BD0255530EF25A030CA23EB25B43082
:10078000CA23D4254930EF25C830CA23EB25DC30F5
:10079000CA23C22884000310780D84070008A4002F
:1007A000840A0008A500A601A701A51FDA2BA5133E
:1007B0002D30EF252E263B3023260800D02549304A
:1007C000C01C5530EF25A030CA23EB25B430CA2316
:1007D000D4250C3079050310CA00CA0CCA0C73303A
:1007E000CA0BF32B5D30CA0BF62B6130CA0BF92B09
:1007F0006E301726EB2503307905CA007830CA0B16
:10080000022C7C30CA0B052C8130CA0B082C863098
:100810001726EB259130791A0E2C8E30F91A112CEF
:100820008B301726EB25CD30D5251724C22841085B
:10083000CA005930CA0B1D2C5D30CA0B202C613008
:1008400017260800D4257808ED25EB25172478080D
:10085000093C031DC22851308A150A1214268A1138
:100860000A124C2440307B1D28304A07E1008A15CB
:100870000A12DA25553014266108043EDA258A1159
:100880000A124108023C0319482CC10A6324C228F9
:10089000FC107C10F024C2284108CA000310CA0DC5
:1008A000CA0DCA0D0800CA0035143518552C780831
:1008B00084000310840D4A08840743088000840ADA
:1008C0004408800008008312031307308A00FC15D7
:1008D0007C16003041070027831603139200831211
:1008E00003139701033041070027CA00CA0C0318FD
:1008F00017164A0C031897163F3995000430C108A3
:100900000319053092000F309704CF30C00541081D
:10091000013C03194016C1080319C01640088500A0
:10092000C1081330031931307D1A31308316031397
:10093000990083120313080007308A00C53042076C
:100940000027CA000608F939CB004A1ACB14CA1A84
:100950004B154B088600F330C005CA1DC0154A1D53
:100960004015400885000800C53042070027CA002E
:10097000F330C005CA1CC0154A1C4015400885004C
:100980000800F9300605CA000C3079050310CB00C9
:10099000CB0CCB0C0301CB0BCE2C0230CB0BD12CD0
:1009A0000430CB0BD42C06304A048600F330C0054B
:1009B00003307905033ACB000310CB0D4B0DC00477
:1009C0004008850008007B088312031790008312FB
:1009D00003134108831203179100831203130800C5
:1009E00083120317100883120313FB0083120317EB
:1009F000110883120313C10063240800F801EF30CB
:100A00008400503083120313C70080018403C70B96
:100A1000052D08000310780DA03EC700A03084000B
:100A200047080402031D192D840A840A1430C707DD
:100A30001D2D8001840A8001840AF0300402031D08
:100A4000102D7D11FD1108008A150A12B125AF2560
:100A50008A110A120A30C700610884000008AC003D
:100A6000840A0008AD00AE01840AAD1F402DAD130D
:100A7000AC09AD09AE09AC0F402DAD0F402DAE0A4B
:100A80002C08A5072D0803182D0FA6072E080318FC
:100A90002E0FA707C70B2E2D8A150A1200206008FB
:100AA0000C268A110A120800831203135930B6006B
:100AB0006230B7000230B800772D83120313033081
:100AC000B6003D30B7000030B800772D8312031315
:100AD0001930B6000630B7000030B800772D831209
:100AE00003133D30B6000030B7000030B800FF30CF
:100AF000B60703180301B70703180301B807031863
:100B00000301360437043804031D772D08000E2630
:100B1000F5010630C6000616861286168612831662
:100B20000313061683120313952D962D972D031488
:100B3000061A0310F50C831603130612831203130F
:100B40000612C60B8D2DF50CF50C75083F39F50016
:100B50000800B51566256625662583120313351131
:100B60000330C7003030C500F3256625C70BB22D12
:100B70002030C500F3256F252830D5250C30D5252C
:100B80000130D5258A110A1626218A110A126F25ED
:100B9000D02508001030D52D0C30D52D0E30D52D98
:100BA0000130D52D0230D52DC030831203133511FD
:100BB000B515C5000310F325F325C50D6F253519AF
:100BC000E52DFC304507031C6625B51108002E30C5
:100BD000EF2D3030EF2D2030EF2D0F3930388312CC
:100BE00003133515D82D0E2606160A26351D0612B6
:100BF0000A2606120A260A260430C6000612C50D69
:100C0000031806160A26C60BFE2D0616072E082EFA
:100C10000612080086160C2E86120800061286128E
:100C20000830C60086168612C60B122E0800C700B2
:100C3000C70307308A0047080027FF390319080057
:100C4000EF25C70A1B2E8400000EED250008ED25B8
:100C500039300402031908008403242E2030BF0019
:100C6000B901BA01BB01BC01BD01A40DA50DA60DC2
:100C7000A70DB90DBA0DBB0DBC0DBD0DBF0B412E9F
:100C800008000530C80039308400472E840A4B26FE
:100C9000C80B462E352E03300007BE00BE1980005B
:100CA00030300007BE00BE1B800008008A150A1203
:100CB00014268A110A125D260800A71F622EA713A8
:100CC0002D30EF25E5010B30E4007E0E0F39E200F8
:100CD00064088A150A122B264C238A110A1200383E
:100CE000031D7D2E0430E407E50A62086502031D3A
:100CF000682E7E080F39E2007F2E0530E20065087D
:100D0000023EE4000310E40DE40D0B3064078A1585
:100D10000A122B26B721E8208A110A122E26B517AF
:100D200049080F39E3003D30CB263D30CB263C301F
:100D3000CB26B51FA12E3C0E0F39031DA12EE92590
:100D4000A32E3C30CB26E3080319B32EE7253B3016
:100D5000BA263B30BA263A30BA263A30BA2639306B
:100D6000BA263930BA263230650700270038031D0D
:100D7000EF2D08008400E20803190800E203E308ED
:100D800003190800800E00080F39031DB513ED2567
:100D9000B51FE30308008400800E0008B51FD42EA1
:100DA0000F3903190800B513E3080319E92DE3030C
:100DB0000008ED25080007308A003E304107E42E88
:0E0DC00007308A003B3041070027FE00080084
:100E000082077C3431340434FA3464340A34A6342E
:100E10006834D434A5349C346E346B342834923422
:100E200074342434003488347A34003400347F3409
:100E30000034003400347534033412346F346B34AE
:100E400006343734BD346134093470345F34573478
:100E50000C34BC34CC344D3410341D347D34433424
:100E600013349234EF3447344D346B3400346D34E2
:100E700002346E3470346634513452345334713425
:100E80007234733452344C34433420344D3465342A
:100E90007434653472342034763431342E3433343F
:100EA00000345234733420340034583473342034D2
:100EB00000343134303430340034203431346B3445
:100EC0000034313430346B3400344F34763465348C
:100ED00072346C346F3461346434003431343034FF
:100EE00030346B3400343134303430340134003435
:100EF000313478343134003431343034783431346E
:100F0000003431347834313430340034783431348E
:100F100030343034003452346534003449346D3464
:100F20000034523449340034433461346C342E3448
:100F3000203400344F34503445344E34003453346C
:100F400048344F345234543400344C344F344134E8
:100F500044342034003453343234203474346F3405
:100F60002034733474346134723474340034733420
:100F70007434643400342D342D342D34003455341D
:100F80002034623469346134733400340C340434F2
:100F90000034103420343034313433347534503428
:100FA0009B348A3472342634E234D4346F340534BA
:100FB00082344434003400340134003400340A34C0
:100FC00000340034643400340334E834003427340B
:100FD000103401348634A0340F3442344034793430
:0E0FE00082346134343498346F34AF343A3490
:101000009630A800A901A71F0E28A509A609A709BF
:10101000A50A0319A60A0319A70AA917B3012708E5
:10102000031D23282608A7002508A600A501B3153F
:101030002708031D23282608A700A601B31133168D
:101040002708031934283308A802031D031C3F2A6C
:101050000310A71B3128A50DA60DA70DA80B292845
:101060003F2AA91FA7130034A701A601A501A401C7
:10107000A80100349E30A800A901A71F4B28A4098D
:10108000A509A609A709A40A0319A50A0319A60A0E
:101090000319A70AA917B3012708031D6B282608FF
:1010A000A7002508A6002408A500A401B315270859
:1010B000031D6B282608A7002508A600A501B3116B
:1010C00033162708031D6B282608A700A601B315B1
:1010D0002708031934283308A802031D031C3F2ADC
:1010E0000310A71B7A28A40DA50DA60DA70DA80B0C
:1010F00071283F2A2A1B251C3128A41F3128A50A44
:101100000319A60A0319A70A031D3128A70CA60C68
:10111000A50CA80A0319AC293128280803190034A2
:101120002708A900A7179630A802A81FDC28A8093D
:10113000A80A08302802031CB828A800A50D260814
:10114000A5002708A600A70108302802031CB8281C
:10115000A800A50D2608A500A60108302802031C3A
:10116000B828A800A50DA5012808031D0310C12853
:1011700028080319C1280310A70CA60CA50CA80B5E
:10118000BB282A1B251CCD28031CCD28A50A031922
:10119000A60A0319A70AA71BDC28A91F0034A70960
:1011A000A609A509A50A0319A60A0319A70A003466
:1011B000A701A601A50100342A14AA1FFF34A70124
:1011C000A91FFF30A700A600A500A90DA70CFF349A
:1011D000A4012808031900342708A900A7179E3086
:1011E000A802A81F4C29A809A80A08302802031C35
:1011F0002129A800A40D2508A4002608A500270879
:10120000A600A70108302802031C2129A800A40D6C
:101210002508A4002608A500A60108302802031C02
:101220002129A800A40D2508A400A5010830280242
:10123000031C2129A800A40DA4012808031D0310E4
:101240002B29280803192B290310A70CA60CA50C81
:10125000A40CA80B24292A1B241C3929031C392976
:10126000A40A0319A50A0319A60A0319A70AA71BAA
:10127000DC28A91F0034A709A609A509A409A40A06
:101280000319A50A0319A60A0319A70A0034A7011E
:10129000A601A501A40100342A14AA1FFF34A70146
:1012A000A91FFF30A700A600A500A400A90DA70C48
:1012B000FF342808031D2F080319342827082E0699
:1012C000A9002F08A8077E30031C6A29A80203186A
:1012D000AC296D29A802031C3F2A2708A400260870
:1012E000A3002508A200A417AE170310A701A601AA
:1012F000A5011830B300221C87292C08A5072D084A
:1013000003182D0FA6072E0803182E0FA707A70CEA
:10131000A60CA50CA40CA30CA20C0310B30B7B29E8
:10132000A71B9729A40DA50DA60DA70DA8032A1B81
:10133000251CA929A41FA929A50A0319A60A03196E
:10134000A70A031DA929A70CA60CA50CA80A031916
:10135000AC29A91FA7130034AA14AA1FFF34FF3019
:10136000A800A700A600A500A90DA70CFF342F0810
:1013700003194A2A28080319342827082E06A90029
:10138000A717AE17B3012708A4002608A300250855
:10139000A2002C08A2022D08031C2D0FA3022E0868
:1013A000031C2E0FA402A401A301A201031CDF2928
:1013B0000310A70CA60CA50CA40C0130B3002F0839
:1013C000A802031CE9297E303307A8070318AC29BB
:1013D000EE297E303307A807031C3F2A1830B200DD
:1013E000A20DA30DA40DA50DA60DA70DB30D2C08E0
:1013F000A5022D08031C2D0FA6022E08031C2E0F7C
:10140000A7022E0DB304331C072A2214122A2C081B
:10141000A5072D0803182D0FA6072E0803182E0A5E
:10142000A7072210B20BF0292A1B221C362A031010
:10143000A50DA60DA70DB30D2C08A5022D08031CA4
:101440002D0FA6022E08031C2E0FA7022E0D33040B
:101450000139A2070318A30A0319A40A031D362A97
:10146000A40CA30CA20CA80A0319AC29A91FA4134D
:101470002408A7002308A6002208A50000342A1586
:10148000AA1FFF340130A800A701A601A501A90DDC
:10149000A70CFF34AA15FF348030AE0627082E06AD
:1014A000B300A401AB0128082F02031C6F2A2F08E8
:1014B000A2002808AF002208A8002E08A2002708D2
:1014C000AE002208A7002D08A2002608AD002208C1
:1014D000A6002C08A2002508AC002208A5002F08B1
:1014E000031900342708A900A717AE172F082802F0
:1014F000AF000319A22A08302F02031C982AAF005C
:101500002C08AB002D08AC002E08AD00AE01083051
:101510002F02031C982AAF002C08AB002D08AC004A
:10152000AD0108302F02031C982A2908A7000034B7
:101530002F080319A22A0310AE0CAD0CAC0CAB0C97
:10154000AF0B9B2AB31FAF2AAB09AC09AD09AE099B
:10155000AB0A0319AC0A0319AD0A0319AE0A2B082A
:10156000A4072C0803182C0FA5072D0803182D0F0E
:10157000A6072E0803182E0FA707B31BC82A031CA3
:101580007A28A70CA60CA50CA40CA80F7A28AC29C5
:1015900003184B28A409A509A609A709A40A031939
:1015A000A50A0319A60A0319A70A8030A9060E285E
:1015B00027082E06B300B31B112BA71BF82A2808F7
:1015C0002F02031C0034031D013427082E02031CC4
:1015D0000034031D013426082D02031C0034031DB2
:1015E000013425082C02031C0034031D013400348F
:1015F0002F082802031C0034031D01342E08270283
:10160000031C0034031D01342D082602031C003482
:10161000031D01342C082502031C0034031D013472
:101620000034AE1F0134003427082E06B300B31B6C
:10163000492BA71B322B28082F02031C0034031D43
:10164000013427082E02031C0034031D0134260830
:101650002D02031C0034031D013425082C02031C39
:10166000003401342F082802031C0034031D013408
:101670002E082702031C0034031D01342D08260206
:10168000031C0034031D01342C082502031C003404
:101690000134AE1F013400342E082706B300B31BFB
:1016A000852BAE1B6C2B2F082802031C0034031D56
:1016B00001342E082702031C0034031D01342D08B9
:1016C0002602031C0034031D01342C082502031CD0
:1016D0000034031D0134003428082F02031C003499
:1016E000031D013427082E02031C0034031D01349E
:1016F00026082D02031C0034031D013425082C028A
:10170000031C0034031D01340034A71F01340034CE
:101710002E082706B300B31BBD2BAE1BA62B2F082C
:101720002802031C0034031D01342E082702031C69
:101730000034031D01342D082602031C0034031D50
:1017400001342C082502031C0034013428082F0220
:10175000031C0034031D013427082E02031C00342F
:10176000031D013426082D02031C0034031D01341F
:1017700025082C02031C00340134A71F0134003457
:101780002F082802031D00342E082702031D0034F1
:101790002D082602031D00342C082502031D0034E9
:1017A00001342F082802031D01342E082702031DCF
:1017B00001342D082602031D01342C082502031DC7
:1017C000013400341C303825243033254E221C309F
:1017D0002C2520303825283033254E2220302C254A
:1017E00008001C303825243033254C221C302C2591
:1017F00020303825283033254C2220302C25080075
:10180000203038252830332559212C302C251C3008
:1018100038252430332559212C3033254C222C30C7
:101820002C2530302C2520303825243033255921E3
:1018300030302C251C3038252830332559213030C4
:1018400033254E2220302C252C3038251C302C25D9
:101850000800243038251026592134302C25283012
:10186000382510265921343033254E2234302C258A
:101870001C3038252430332559212C302C2520309C
:1018800038252830332559212C3033254E22343049
:101890003325B7212C302C251C3038252830332512
:1018A000592130302C25243038252030332559213A
:1018B000303033254C2234303325B72120302C25CD
:1018C0002C3038251C302C2508008A110A124C2493
:1018D000CA0DCA0DCA0D4208CB000310CB0DCB0DAB
:1018E000CB0D04304A074B078A150A1208008A11EB
:1018F0000A124C2428304A078A150A1208008A1155
:101900000A124C2440304A078A150A120800831232
:101910000313E6001C30902C83120313E6002430DE
:10192000033E84000230C70083170430C800CB2573
:10193000800083120313E60A8403C80B972CC70B9D
:10194000A32C8313080008308407952CCD001F308A
:10195000AB2CCD002730C82416308A004D08002655
:101960008A150A12CE24C70BAC2C83130800CD00B5
:101970001F30BC2CCD002730C82417308A004D08FA
:1019800000278A150A12CE24C70BBD2C831308002A
:1019900083178400CD030830C70008008000CD0AFB
:1019A00084034708053C08300319840708008312A4
:1019B00003178D0034308E00831203130830C700E4
:1019C00083171F3084000008831203178C008403E0
:1019D000831603178C170C158B1355308D00AA3006
:1019E0008D008C14000000000C118B17831203175C
:1019F0008D0A831203134708053C08300319840736
:101A0000C70BE32C83120313831308008312031301
:101A1000CA001C30CB0088303E2D83120313CB004C
:101A20001C30162D83120313CB002430CA0048301B
:101A30003E2D83120313CB001C30CA002A2D8312C3
:101A40000313CB002430CA002A2D83120313CA00CB
:101A50001C30CB00C8303E2D83120313CA00253042
:101A6000CB0044303E2D83120313CB002C303C2D91
:101A700083120313CB002530CA008430E8000F30F6
:101A80006805C7004B0884008313E81B8317000810
:101A9000CC004A0884004C088313681B831780001D
:101AA000CA0ACB0AC70B422D83130800FD1A7E2DEC
:101AB0006524B72477248C24F123403025257F2406
:101AC00087244E301225F12340301F25002440305A
:101AD00025257F2487246524BA24F1233830252541
:101AE0004E300D2577248C24F12338301F25002417
:101AF00040301F2529246524A924002496257B1D18
:101B00008B2D24302525173026261C302C25B12579
:101B100020302C2529244E30062508004E300D2576
:101B20005630122529244E30062508007D1C9A2D9A
:101B3000F9170800FD1C9E2DF9130800F917203035
:101B40003825EF302B264C23003803190800F330DA
:101B50002B26D822003803190800F91308002F306B
:101B6000B22D283084000430C70080018403C70BE5
:101B7000B52D0800E6002830BF2DE6002F30840088
:101B80000430C700CB25831203138000E60A8403C8
:101B9000C70BC22D08006608831203178D00831639
:101BA00003178C130C14831203170C080800E600AB
:101BB0002F30DC2DE600283084000430C7000008F8
:101BC000E700EF2583120313E60A8403C70BDF2D1A
:101BD000831603178C18EA2D83120313080083164B
:101BE00003178C18F12D8312031366088312031751
:101BF0008D00831203136708831203178C0083166A
:101C000003178C130C158B1355308D00AA308D00E3
:101C10008C148B170C110800CA002830CB00172E2B
:101C20002830CB002F30162ECB002830CA000430CD
:101C3000C7004B0884000008CC004A0884004C0808
:101C40008000CA03CB03C70B192E0800CD00CD03BB
:101C5000283084002F2ECD00CD032F308400043097
:101C6000C7008A110A1207308A004D0800278A151A
:101C70000A128000CD0A8403C70B312E0800CA0067
:101C80000310CA0DCA0D08004C26C9009626C90EBD
:101C9000C904610BC90E0800A03084000310780D40
:101CA000742685266508E3006408E2001330742674
:101CB00085266308E1006208E00085266008A4002C
:101CC0006108A500A601A7018A110A122E268A150D
:101CD0000A12BB08031D0534F0303A05031D043415
:101CE000BA08031D0334023484070008E000840AA4
:101CF0000008E100133084070008E400840A0008AB
:101D0000E5007F30E105E505080060086402610830
:101D1000031C610F65020318080061086502E107F2
:101D2000E50260086402E007E4020800E1015130C6
:101D30001426553011267F30A705AE0588230038BC
:101D4000031DAA2EE10A55301426513011267F308A
:101D5000A705AE05B7210038031D023413302B262A
:101D600088230038031D0234BB264902023C0318B5
:101D70000234023C0800E8208A110A122E268A1535
:101D80000A12BA08031D0234F0303905031D01346C
:101D9000003418307C050319D02E0830FC020800EE
:101DA0001F151F19D12EB125831603131E08831288
:101DB0000313A5001E08A60000202030BD255921D0
:101DC00010269830BA2500205921E8208A110A12DD
:101DD0002E268A150A12BA08031DF22E0330390284
:101DE000031C08008A110A128B30D5250330E3004A
:101DF000B517BA0E3A30CB268C30D525B51339300D
:101E0000CB26E7253930CB265630EF258A150A1226
:021E10000800C8
:10200000CA000830CA0710300318013E8A004A0887
:10201000820000340E341134113411340A341B346C
:102020000034003400341234123412341E341134AB
:10203000103400340134033407340F3407340334CC
:102040000134003408340C340E340F340E340C34A4
:1020500008340034043404340E340E341F341F3476
:10206000003400341F341F340E340E34043404346E
:1020700000340C3414341C34143400340034003470
:10208000003498004930980710300318013E8A0048
:1020900018088200533465347434743469346E34EF
:1020A00067347334003452346534733465347434B3
:1020B000203474346F34203464346534663400342E
:1020C0004534643469347434003401340A341734C8
:1020D00020344534733463342034203403342034C2
:1020E000203404342034203445346E3474342034A5
:1020F0000034453420342034033420342034063472
:102100002034203405342034203404342034203466
:102110004E3400344E3465346534643420346334D2
:1021200061346C342E3420344C344F3441344434D4
:102130002034003420344F344B340034083402341B
:102140000334533461347634653420346134753467
:1021500074346F340034533461347634653420344D
:102160006E346F347734003453346F3475346E34D6
:10217000643420346F346E34003453346F34753427
:102180006E34643420346F34663466340034413441
:102190004434433420343234353430346B344834AE
:1021A0007A340034413444344334203431343034CC
:1021B00030346B3448347A3400344F3453344C3434
:1021C00020346F346E3400344F3453344C34203464
:1021D0006F346634663400344F34703465346E3492
:1021E0002F34533468346F347234743400345334BD
:1021F00065347434743469346E3467347334003441
:10220000523473347434643400344C342F344334D3
:10221000733474346434003443346F346534663456
:102220006634203455342034623469346134733474
:102230000034583462346B3474347E3489349434CA
:102240009B34A334AE34B734BC34C33448308A1121
:102250000A12D5258A110A16C701C70A47080020A5
:102260008A110A12EF258A110A16C70A3930470265
:10227000031D2E2908008A110A12EF258A110A1659
:102280008312031708008A110A12EF25EB258A1121
:102290000A168312031708009A009B011A084120AE
:1022A000FF39031957293B219A0A9B0A4E291B081B
:1022B00008009A009B011A084120FF39031963297D
:1022C0009A0A9B0A5B291B0808009A001A0803193E
:1022D00008008A110A12EB258A110A1683120317C5
:1022E0009A0B692908001507412093005921103CD9
:1022F00099000310190C9900652113084C21190746
:10230000103C6521080083120313FB1C9429351A25
:1023100087298B13351683160313833081008312AC
:1023200003131430FA008B1783120313080083126F
:1023300003138A110A125D258A110A1683120317E4
:1023400008008312031792018A110A12D4258A11F8
:102350000A16831203171F304C21033096001C30DD
:1023600095008A110A12D2258A110A1683120317C0
:102370001208732197213F3076020319EC29761950
:10238000C9293F30F60003309208031992009203E6
:10239000B129F619D3293F30F600920A0330120210
:1023A00003199201B129F618DA29831203138A114D
:1023B0000A12B329761AEC293F30F6008A110A1264
:1023C000D2258A110A16831203171C3012074120E6
:1023D0004C21103C6521EF293F30F600BA299401C9
:1023E0008A110A12D4258A110A16831203171208B9
:1023F0009A0055309B00031097011A080319062A0A
:102400001B08412097079B0A9A03FD29D030170724
:10241000950055301207412096008A110A12D425E2
:102420008A110A1683120317140873214222831299
:10243000031797213F30760203193F2A7619282A7D
:102440003F30F600160894080319940094030D2AEF
:10245000F619322A3F30F600940A160814020319BE
:1024600094010D2AF618372A3F30F600A429761A6F
:102470003F2A3F30F60017081407013E852A3F30F7
:10248000F600192A17081407013E98004F309807E4
:1024900012300318013E8A001808831203138200C9
:1024A0005D2A602A632A662A692A6C2A6F2A722AA0
:1024B000080008000800080008007B1E0800752AB4
:1024C0007B1A0800752AFB1C0800752AFB180800F7
:1024D000752A7D1A0800752A7D1E0800752AFD1AC6
:1024E0000800752AFD1E0800752A83120317BF30E5
:1024F0001907831203138A110A12D5252A30EF25F2
:102500008A110A1683120317080098008F30980763
:1025100012300318013E8A00180883120313820048
:102520009D2AA02AA32AA62AA92AB12AB32AB62A12
:10253000B92ABB2A232B202B1D2B7B160523BD2A52
:102540007B120523BD2AFB140323BD2AFB100323A2
:10255000BD2A7D128A110A1263248A110A160323E6
:10256000BD2A7D16AA2AFD120323BD2AFD160323C8
:10257000BD2AD822BD2AEA22BD2A8A110A12D425F0
:102580008A110A16831203171408150741204C21DB
:10259000930051304C211307103C65218312031323
:1025A0008A110A125425542554258A110A16A42981
:1025B0008A150A12B1252830CA004A088A150A125B
:1025C000DA258A110A160430CA074A08583C031D46
:1025D000DD2A08000330FB000130C100FD010523A6
:1025E000FD2A9C308A150A12BA25280801387F393D
:1025F000FB002708C1002608FD008A110A12632487
:102600008A110A1608007B1E08009C30E6007B0831
:10261000E7008A150A12EF2583120313E60A410820
:10262000E700EF2583120313E60A7D08E700EF2594
:10263000831203138A110A1608009830E000262B33
:102640005C30E000252B5830E0005C248A150A122B
:10265000BD252F08DF00E1018A110A12E324CE25EF
:10266000D025D4258A110A168312031730304C2145
:1026700083120313F223BC233F3076020319B42BD9
:10268000791F442B7913B42BB51C552BB510F61AB2
:10269000B42B5F1F4D2B8630502BDF1FB42B4830DF
:1026A000DF00F223BC237C15B42B7618602B7C1939
:1026B0001E248A110A12CC25F0248A110A16A42994
:1026C000F618692BE10A073061020319E1011224AF
:1026D000B42B7619772B7C15452470246524A71F0D
:1026E0008A150A1210268A110A16BC23B42BF61971
:1026F000932B452465242708983C031C912B031D2C
:102700008B2B2608963C031C912B031D8B2B250835
:102710007F3C031C912B7C158A150A1210268A1106
:102720000A16BC23B42B761A9D2BE103FF306102FD
:1027300006300319E1001224B42BF61AB42B7C19CD
:102740001E24DF080319592BC20A0830420203195C
:10275000C2015C248A150A12BD252F08DF008A11E8
:102760000A16F223BC23B42B3F30F6008A110A125A
:102770005D258A110A163C2BA801A7012C08A4008C
:102780002D08A5002E08A6008A110A128630D5252C
:102790002E26B5130830E300BC0E3C30CB263B3070
:1027A000CB263B30CB26E7253A30CB263A30CB261A
:1027B0003930CB263930CB268A110A16DF080319A7
:1027C000F02B8A110A125F030F39E500B32601309E
:1027D0005F1B4630DF1B4830EF25EB258A110A16B8
:1027E000122408008A110A128030D5258A110A168F
:1027F000DF08031D022C8A110A12BF3017268A1126
:102800000A1608008A110A1252305F1B4330DF1B80
:102810004C30EF25B73017264208ED25EB258A11FD
:102820000A1608000430610261080318013E8A118B
:102830000A128D3CD5258A110A1608007C115F0802
:10284000AF009830DF08031D5C248A150A12D725D3
:102850008A110A16DF08031D7B248A110A128030B0
:10286000D5258A110A168312031741304C21831291
:1028700003138A110A124208ED25542554255425C4
:1028800054258A110A1641250800A801A70107301E
:102890008A000310610D6107D93ECA008A110A122D
:1028A0000027A700CA0A4A080027A6004A0A0027EC
:1028B000A5008A110A1608004208CA000310CA0DB2
:1028C000CA0DCA0D60084A0708002C08A5072D0884
:1028D00003182D0FA6072E0803182E0FA7070800B0
:1028E00083120313A509A609A709A50A0319A60AB5
:1028F0000319A70A08005C24DE00C0305F0504301D
:10290000031DDE025E088A150A12BA252808DF00B8
:10291000A80100202430BD25B7215F083F260B30D9
:102920004A072B26592138302C2510261730262609
:10293000B7213C302C2504305E07BA252808DF007B
:10294000A80100202430BD25B7210F305F053F26A8
:102950000B304A072B26592140302C25C1018A15FE
:102960000A1241083F26CE304A072B264030382530
:10297000B7218A110A165F1FE72C8A150A12283020
:102980002C253C30382524302C25173026261C30A9
:102990002C25B12520302C2529248A150A128312D2
:1029A000031716308F00831203136524D724831274
:1029B000031717308F00831203136524D7248A115D
:1029C0000A16C10A03304102031DAF2C08008A1504
:1029D0000A1220302C25383038251C302C258A113D
:1029E0000A16CD2C8A110A12D4257808ED25EB257C
:1029F00017247808093C031DC2288A150A128E255F
:102A00008312031717308F00831203136524D72412
:102A10008A110A164108023C0319132DC10A8A11B2
:102A20000A126324C2287C13FC1236258A110A126A
:102A3000F024C2282525E405031D08008A110A1286
:102A4000CD30D5252130EF250800420AE5000314DA
:102A5000E401E40DE50B292D9F30E6008A150A12EA
:102A6000CB25831203138A110A1608002525640456
:102A7000E7009F30E6008A150A12EF258312031340
:0C2A800008002525E50064096505382DD7
:102C000082070000000000007F34003400340034EC
:102C10006C345234D43424348234203400340034BC
:102C20006C345234D4342434863448340034003480
:102C30006C345234D434243489347A34003400343B
:102C40007234D234D43427348D341C3440340034BC
:102C50007934A434B534BE34903443345034003421
:102C600080348034AD34FC349334743424340034F0
:102C70008634C9340F34DA349634183496348034B8
:102C80008B349D34143462347F3400340034003487
:102C900070340334C4349834823420340034003423
:102CA00070340334C43498348634483400340034E7
:102CB00070340334C434983489347A3400340034A2
:102CC00076348334C43498348D341C344034003426
:102CD0007C34CD34E3342E349034433450340034D7
:102CE0008334A034D9347C34933474342334F034B2
:102CF0008934FB345334C0349634183495348434D6
:102D00008E34C434583438347F34003400340034C2
:102D100073342434B534BC34823420340034003469
:102D200073342434B534BC3486344834003400342D
:102D300073342434B534BC3489347A3400340034E8
:102D40007934A434B534BF348D341C344034003469
:102D500080348034AD34FD34903443344F34F43413
:102D60008634C9340F34CE34933474341D34AF34C4
:102D70008D349D34103452349634183434340E3437
:082D80009134F434D1348234A3
:102E000082070000000000007F34003400340034EA
:102E10006C345234D43424348234203400340034BA
:102E20006C345234D434243486344834003400347E
:102E30006C345234D434243489347A340034003439
:102E40007234D234D43427348D341C3440340034BA
:102E50007934A434B534BE3490344334503400341F
:102E600080348034AD34FC349334743424340034EE
:102E70008634C9340F34DA349634183496348034B6
:102E80008B349D34143462347F3400340034003485
:102E900070340334C4349834823420340034003421
:102EA00070340334C43498348634483400340034E5
:102EB00070340334C434983489347A3400340034A0
:102EC00076348334C43498348D341C344034003424
:102ED0007C34CD34E3342E349034433450340034D5
:102EE0008334A034D9347C34933474342334F034B0
:102EF0008934FB345334C0349634183495348434D4
:102F00008E34C434583438347F34003400340034C0
:102F100073342434B534BC34823420340034003467
:102F200073342434B534BC3486344834003400342B
:102F300073342434B534BC3489347A3400340034E6
:102F40007934A434B534BF348D341C344034003467
:102F500080348034AD34FD34903443344F34F43411
:102F60008634C9340F34CE34933474341D34AF34C2
:102F70008D349D34103452349634183434340E3435
:082F80009134F434D1348234A1
:02400E00723FFF
:104200007F0000000000000082002000000000008D
:10421000850048000000000088007A0000000000CF
:104220008C001C00400000008F0043005000000084
:104230009200740024000000960018009600800090
:1042400070007900DB002200823420340034003416
:10425000000000000000000000000000000000005E
:10426000000000000000000000000000000000004E
:10427000000000000000000000000000000000003E
:10428000000000000000000000000000000000002E
:10429000000000000000000000000000000000001E
:1042A000000000000000000000000000000000000E
:1042B000040000002700100086000000000032000B
:1042C000040001008600A00086000000000032000B
:1042D00004001E0084008000860000000000320000
:1042E000030000004E0020004800000003002000F2
:1042F000030003000D004000480000000300200000
:1043000003001E008400800048000000030020001D
:10431000020000004E0020004800000003002000C2
:10432000020001008600A0004800000003002000F9
:104330000000000027001000030001000000000042
:00000001FF
